:020000040000FA
:0400000000003329A0
:08000800A000030E8312A10009
:100010000A08A2000408A3008C1CD3288C103A08FC
:10002000B906BA0905083B06BA05B905FF3A39040D
:100030003A04FF3ABC00BB063C1C28283B1C28287D
:10004000BD01BE01BF014908B2000130B100332833
:10005000BC1D3328BB193328BD01BE01BF014908AF
:10006000B2000430B10000308A00310882076928EC
:100070003C283E288F2840284030412843304128E2
:10008000463084000008BF07031C4B28BE0F4B28D6
:10009000BD0A03195828840A0008BE07031C532808
:1000A000BD0A03195828840A0008BD07031C6028EC
:1000B000BD01BE01BF01B10A3108053A0319B10102
:1000C00000308A003108820769286C287E288F2832
:1000D0009328CB01CC01C9283209AC003D08071A8E
:1000E0007728BE21A8003D0ABE21A9000021DC20FE
:1000F00032082D07C9002E08CA00A5283509AC0012
:100100003D08071A8928C622A8003D0AC622A90070
:100110000021DC202D09C9002E09CA00A5283508B8
:10012000C900CA01A5283208AC003D08071A9E285C
:10013000C622A8003D0AC622A9000021DC203209FF
:100140002D07FF3AC9002E09CA00CB01CC0138089F
:1001500003104918CB07CB0CCC0CC918CB07CB0C20
:10016000CC0C4919CB07CB0CCC0CC919CB07CB0C49
:10017000CC0C491ACB07CB0CCC0CC91ACB07CB0C37
:10018000CC0C491BCB07CB0CCC0CC91BCB07CB0C25
:10019000CC0CCC0D9516031C9512CC0D1516031C1A
:1001A00015124B08930022088A0023088400210EB0
:1001B0008300A00E200E0900AD01AE0103102C1823
:1001C000AD07AD0CAE0CAC18AD07AD0CAE0C2C19D8
:1001D000AD07AD0CAE0CAC19AD07AD0CAE0C2C1AC6
:1001E000AD07AD0CAE0CAC1AAD07AD0CAE0C2C1BB4
:1001F000AD07AD0CAE0CAC1BAD07AD0CAE0C0800E2
:100200002808A902AA01AB01290803103E18AA0771
:10021000AA0CAB0CBE18AA07AA0CAB0C3E19AA0775
:10022000AA0CAB0CBE19AA07AA0CAB0C3E1AAA0763
:10023000AA0CAB0CBE1AAA07AA0CAB0C3E1BAA0751
:10024000AA0CAB0CBE1BAA07AA0CAB0C28082A07E9
:1002500008000630A400A40B2B299F149F182E29F8
:100260001E08B00008008701073099009101043092
:1002700092009301831602308C00F63091002030FA
:100280009F00FF3092001F3087003F3085009601AD
:10029000831200308C00C0308B000C309500B3010D
:1002A000B401B501B6018030B700FF30B800B1012C
:1002B000BF01BE01BD01C001C101C201C301C40132
:1002C000C501C601C701C801C901CA01CB01CC01E2
:1002D0000730AF00B201B901BA01BB01BC01AF0ADE
:1002E00001308A002F08073982077D298D299D2931
:1002F000A229B229B929AF0A6F2905309F00292107
:10030000B30037083302031C0030A600CE23C2001E
:10031000D524C100DC25C0006F2909309F002921A8
:10032000B40037083402031C0030A600CE23C500F9
:10033000D524C400DC25C3006F2911309F0029217A
:10034000B5006F2915309F002921B6003708360205
:10035000031C0030A600CE23C800D524C700DC252E
:10036000C6006F2919309F002921B7000310B70C70
:100370006F291D309F002921B8006F29A500013089
:100380008A002508C63E03188A0A82000034013418
:1003900003340534073409340B340D340E3410346F
:1003A000123414341634173419341B341D341E34EB
:1003B0002034223423342534273429342A342C346D
:1003C0002D342F34313432343434363437343934F4
:1003D0003A343C343D343F3441344234443445347F
:1003E000473448344A344B344C344E344F3451340F
:1003F0005234543455345734583459345B345C34A3
:100400005D345F346034623463346434663467343A
:10041000683469346B346C346D346F3470347134D7
:100420007234743475347634773479347A347B3476
:100430007C347D347E34803481348234833484341B
:1004400085348734883489348A348B348C348D34C1
:100450008E348F349034923493349434953496346B
:100460009734983499349A349B349C349D349E3418
:100470009F34A034A134A234A334A434A534A634C8
:10048000A734A834A934AA34AA34AB34AC34AD347C
:10049000AE34AF34B034B134B234B334B334B43432
:1004A000B534B634B734B834B934B934BA34BB34EB
:1004B000BC34BD34BE34BE34BF34C034C134C234A5
:1004C000C234C334C434C534C634C634C734C83463
:1004D000C934C934CA34CB34CC34CC34CD34CE3422
:1004E000CE34CF34D034D134D134D234D334D334E5
:1004F000D434D534D534D634D734D834D834D934A8
:10050000DA34DA34DB34DB34DC34DD34DD34DE346D
:10051000DF34DF34E034E134E134E234E234E33434
:10052000E434E434E534E534E634E734E734E834FD
:10053000E834E934E934EA34EB34EB34EC34EC34C9
:10054000ED34ED34EE34EE34EF34EF34F034F03497
:10055000F134F234F234F334F334F434F434F53463
:10056000F534F634F634F734F734F834F834F93433
:10057000F934F934FA34FA34FB34FB34FC34FC3407
:10058000FD34FD34FE34FE34FF34FF34A500023068
:100590008A002508CE3E03188A0A820000340734F8
:1005A0000E3414341B34213428342E34343439348A
:1005B0003F34443449344F34533458345D34623416
:1005C00066346A346E34723476347A347E348234EB
:1005D000853489348C348F349234953498349B34F8
:1005E0009E34A134A334A634A834AB34AD34B03433
:1005F000B234B434B634B834BA34BC34BE34C03493
:10060000C234C334C534C734C834CA34CB34CD340F
:10061000CE34D034D134D234D334D534D634D734A4
:10062000D834D934DA34DB34DC34DD34DE34DF344E
:10063000E034E134E234E334E434E434E534E63401
:10064000E734E734E834E934E934EA34EA34EB34C3
:10065000EC34EC34ED34ED34EE34EE34EF34EF348E
:10066000F034F034F134F134F134F234F234F33460
:10067000F334F334F434F434F434F534F534F53439
:10068000F534F634F634F634F734F734F734F73417
:10069000F734F834F834F834F834F934F934F934F8
:1006A000F934F934F934FA34FA34FA34FA34FA34DD
:1006B000FA34FB34FB34FB34FB34FB34FB34FB34C3
:1006C000FB34FC34FC34FC34FC34FC34FC34FC34AB
:1006D000FC34FC34FC34FD34FD34FD34FD34FD3495
:1006E000FD34FD34FD34FD34FD34FD34FD34FD3482
:1006F000FD34FE34FE34FE34FE34FE34FE34FE346B
:10070000FE34FE34FE34FE34FE34FE34FE34FE3459
:10071000FE34FE34FE34FE34FE34FE34FE34FE3449
:10072000FE34FE34FF34FF34FF34FF34FF34FF3433
:10073000FF34FF34FF34FF34FF34FF34FF34FF3421
:10074000FF34FF34FF34FF34FF34FF34FF34FF3411
:10075000FF34FF34FF34FF34FF34FF34FF34FF3401
:10076000FF34FF34FF34FF34FF34FF34FF34FF34F1
:10077000FF34FF34FF34FF34FF34FF34FF34FF34E1
:10078000FF34FF34FF34FF34FF34FF34FF34FF34D1
:10079000FF34FF34FF34FF34FF34FF3403308A006A
:1007A0002608D53E03188A0A82000C340C340B3418
:1007B0000B340B340A340A3409340934093408344C
:1007C0000834083408340734073407340634063450
:1007D000063406340634053405340534053405344E
:1007E000043404340434043404340434033403344B
:1007F0000334033403340334033403340234023443
:100800000234023402340234023402340234023438
:10081000023401340134013401340134013401342F
:100820000134013401340134013401340134013420
:100830000134013401340134003400340034003414
:100840000034003400340034003400340034003408
:1008500000340034003400340034003400340034F8
:1008600000340034003400340034003400340034E8
:1008700000340034003400340034003400340034D8
:1008800000340034003400340034003400340034C8
:1008900000340034003400340034003400340034B8
:1008A00000340034003400340034003400340034A8
:1008B0000034003400340034003400340034003498
:1008C0000034003400340034003400340034003488
:1008D0000034003400340034003400340034003478
:1008E0000034003400340034003400340034003468
:1008F0000034003400340034003400340034003458
:100900000034003400340034003400340034003447
:100910000034003400340034003400340034003437
:100920000034003400340034003400340034003427
:100930000034003400340034003400340034003417
:100940000034003400340034003400340034003407
:1009500000340034003400340034003400340034F7
:1009600000340034003400340034003400340034E7
:1009700000340034003400340034003400340034D7
:1009800000340034003400340034003400340034C7
:1009900000340034003400340034003400340034B7
:1009A0000034003400340034003404308A00260857
:1009B000DC3E03188A0A8200CC345934E9347D3491
:1009C0001534B1345034F33499344234EE349D3418
:1009D0004F340434BC3476343234F134B2347634A7
:1009E0003B340334CC349834653434340534D8344F
:1009F000AC348234593432340C34E734C434A23445
:100A000081346134433425340934ED34D334B9347A
:100A1000A034893472345C34463432341E340B349E
:100A2000F834E634D534C434B434A5349634883438
:100A30007A346D346034533447343C3430342634A3
:100A40001B3411340834FE34F534ED34E434DC3432
:100A5000D434CD34C634BF34B834B134AB34A53417
:100A60009F34993494348F348A34853480347C3480
:100A7000773473346F346B346734633460345D348B
:100A800059345634533450344D344A344834453450
:100A9000433440343E343C343A34383436343434DD
:100AA000323430342E342D342B342A342834273445
:100AB000253424342334213420341F341E341D348F
:100AC0001C341B341A3419341834173416341634C1
:100AD00015341434133413341234113411341034E3
:100AE0000F340F340E340E340D340D340C340C34FA
:100AF0000B340B340B340A340A3409340934093406
:100B0000083408340834083407340734073406340A
:100B10000634063406340634053405340534053409
:100B20000534043404340434043404340434033405
:100B300003340334033403340334033403340234FE
:100B400002340234023402340234023402340234F5
:100B500002340234013401340134013401340134EB
:100B600001340134013401340134013401340134DD
:100B700001340134013401340134003400340034D0
:100B800000340034003400340034003400340034C5
:100B900000340034003400340034003400340034B5
:100BA00000340034003400340034003400340034A5
:100BB000003400340034003405308A002608E33E57
:100BC00003188A0A8200CC3400344C348A349734B7
:100BD00050349534453440346B34A634D834E4343E
:100BE000B23428342E34AE349034BF342634B13489
:100BF0004E34E8346F34D034FB34E03470349A34FB
:100C0000513486342C3437349834453432345334A8
:100C10009D34063484340D3497341A348C34E634DD
:100C20001E342E340D34B4341D34403416349A340A
:100C3000C5349134F934F7348634A13442346634FF
:100C400006342034AF34AE341934EE342734C23491
:100C5000BB340E34BA34B9340A34AA349534CA34A5
:100C60004534043404344434C13479346A3491341E
:100C7000EE347D343E342E344C3496340B34A93467
:100C80006E345A346A349F34F5346D340534BB34D1
:100C90008F3480348D34B434F5344F34C1344A3415
:100CA000E9349E3467344534363439344F3475343E
:100CB000AD34F4344C34B2342734A9343934D73415
:100CC00080343634F734C4349C347E346A3460342F
:100CD0005F34673479349234B434DD340E344734BD
:100CE0008634CD341A346D34C63425348A34F43421
:100CF0006434D9345334D1345434DB346734F73466
:100D00008B342234BD345C34FE34A4344D34F93495
:100D1000A73459340E34C5347E343B34F934BA34F4
:100D20007D3443340A34D3349F346C343B340B3435
:100D3000DE34B23487345E3437341034EC34C834A3
:100D4000A63485346534463429340C34F134D63431
:100D5000BC34A3348C3475345E3449343434203498
:100D60000D34FA34E934D734C734B634A734983460
:100D70008A347C346E346134553449343D343234F1
:100D800027341D3412340934FF34F634EE34E5349C
:100D9000DD34D534CE34C634BF34B934B234AC3497
:100DA000A634A0349A3495348F348A34853481340F
:100DB0007C34783473346F346B3468346434603426
:060DC0005D345A34563484
:02400E00C230BE
:00000001FF
